
 DDEML

 Start     Length     Name                   Class
 0001:0000 000CAH     INIT_TEXT              CODE
 0002:0000 07E20H     _TEXT                  CODE
 0003:0000 00010H     NULL                   BEGDATA
 0003:0010 00174H     _DATA                  DATA
 0003:0184 00000H     CDATA                  DATA
 0003:0184 00000H     XIFB                   DATA
 0003:0184 00000H     XIF                    DATA
 0003:0184 00000H     XIFE                   DATA
 0003:0184 00000H     XIB                    DATA
 0003:0184 00000H     XI                     DATA
 0003:0184 00000H     XIE                    DATA
 0003:0184 00000H     XPB                    DATA
 0003:0184 00000H     XP                     DATA
 0003:0184 00000H     XPE                    DATA
 0003:0184 00000H     XCB                    DATA
 0003:0184 00000H     XC                     DATA
 0003:0184 00000H     XCE                    DATA
 0003:0184 00000H     XCFB                   DATA
 0003:0184 00000H     XCF                    DATA
 0003:0184 00000H     XCFE                   DATA
 0003:0184 0000CH     DBDATA                 DATA
 0003:0190 00000H     CONST                  CONST
 0003:0190 00019H     HDR                    MSG
 0003:01A9 00082H     MSG                    MSG
 0003:022B 00002H     PAD                    MSG
 0003:022D 00001H     EPAD                   MSG
 0003:0230 00000H     _BSS                   BSS
 0003:0230 00000H     XOB                    BSS
 0003:0230 00000H     XO                     BSS
 0003:0230 00000H     XOE                    BSS
 0003:0230 0001CH     c_common               BSS

 Origin   Group
 0003:0   DGROUP

 Address   Export                  Alias

 0002:4A20 CLIENTWNDPROC           CLIENTWNDPROC
 0002:5C46 CONVLISTWNDPROC         CONVLISTWNDPROC
 0002:1F86 DDEABANDONTRANSACTION   DDEABANDONTRANSACTION
 0002:1BAC DDEACCESSDATA           DDEACCESSDATA
 0002:189A DDEADDDATA              DDEADDDATA
 0002:14B6 DDECLIENTTRANSACTION    DDECLIENTTRANSACTION
 0002:1F3A DDECMPSTRINGHANDLES     DDECMPSTRINGHANDLES
 0002:0C0E DDECONNECT              DDECONNECT
 0002:07EE DDECONNECTLIST          DDECONNECTLIST
 0002:17EA DDECREATEDATAHANDLE     DDECREATEDATAHANDLE
 0002:1D08 DDECREATESTRINGHANDLE   DDECREATESTRINGHANDLE
 0002:0CA8 DDEDISCONNECT           DDEDISCONNECT
 0002:0BA8 DDEDISCONNECTLIST       DDEDISCONNECTLIST
 0002:2186 DDEENABLECALLBACK       DDEENABLECALLBACK
 0002:1CA0 DDEFREEDATAHANDLE       DDEFREEDATAHANDLE
 0002:1DCA DDEFREESTRINGHANDLE     DDEFREESTRINGHANDLE
 0002:1AB2 DDEGETDATA              DDEGETDATA
 0002:17A6 DDEGETLASTERROR         DDEGETLASTERROR
 0002:0010 DDEINITIALIZE           DDEINITIALIZE
 0002:1E36 DDEKEEPSTRINGHANDLE     DDEKEEPSTRINGHANDLE
 0002:22DC DDENAMESERVICE          DDENAMESERVICE
 0002:12B0 DDEPOSTADVISE           DDEPOSTADVISE
 0002:3362 DDEPOSTHOOKPROC         DDEPOSTHOOKPROC
 0002:0F06 DDEQUERYCONVINFO        DDEQUERYCONVINFO
 0002:0AAC DDEQUERYNEXTSERVER      DDEQUERYNEXTSERVER
 0002:1EA0 DDEQUERYSTRING          DDEQUERYSTRING
 0002:0D40 DDERECONNECT            DDERECONNECT
 0002:326E DDESENDHOOKPROC         DDESENDHOOKPROC
 0002:11B8 DDESETUSERHANDLE        DDESETUSERHANDLE
 0002:1C48 DDEUNACCESSDATA         DDEUNACCESSDATA
 0002:044E DDEUNINITIALIZE         DDEUNINITIALIZE
 0002:5A7E DMGWNDPROC              DMGWNDPROC
 0002:663E EmptyQTimerProc         EmptyQTimerProc
 0002:73DE INITENUM                INITENUM
 0002:389C MONITORWNDPROC          MONITORWNDPROC
 0002:571C SERVERWNDPROC           SERVERWNDPROC
 0002:59AC SUBFRAMEWNDPROC         SUBFRAMEWNDPROC
 0002:040A TERMDLGPROC             TERMDLGPROC
 0001:0034 WEP                     WEP

  Address         Publics by Name

 0002:2050       ABANDONTRANSACTION
 0002:2956       ADDADVLIST
 0002:27A0       ADDHWNDHSZLIST
 0002:2DD8       ADDPILEITEM
 0002:66EC       ADDQI
 0002:50FC       ADVANCEXACTION
 0002:605C       ALLOCDDESEL
 0002:383C       ALLOCMONBUF
 0003:00AC       APROGMANHACK
 0003:00AE       AULMAPTYPE
 0000:0000  Imp  BITBLT               (GDI.34)
 0000:0000  Imp  CALLMSGFILTER        (USER.123)
 0003:0026       CCDEF
 0002:52F4       CHECKCBQ
 0002:5A12       CHILDMSG
 0002:2AA6       CLEANUPADVLIST
 0002:71F8       CLIENTCREATE
 0002:78F2       CLIENTINITACK
 0002:4A20       CLIENTWNDPROC
 0002:398C       CLIENTXFERREQ
 0002:4764       CLIENTXFERRESPOND
 0003:0038       CMONITOR
 0002:285E       CMPADV
 0002:25DA       CMPDWORD
 0002:2620       CMPHIWORD
 0002:2602       CMPWORD
 0002:5C46       CONVLISTWNDPROC
 0002:6EB2       COPYBITMAP
 0002:6E60       COPYDDESHAREHANDLE
 0002:7022       COPYHDDEDATA
 0002:2F62       COPYHUGEBLOCK
 0000:0000  Imp  COPYMETAFILE         (GDI.151)
 0002:6F8A       COPYPALETTE
 0002:28EE       COUNTADVREQLEFT
 0000:0000  Imp  CREATECOMPATIBLEBITMAP (GDI.51)
 0000:0000  Imp  CREATECOMPATIBLEDC   (GDI.52)
 0002:24BC       CREATELST
 0000:0000  Imp  CREATEPALETTE        (GDI.360)
 0002:2C10       CREATEPILE
 0002:6666       CREATEQ
 0002:77CA       CREATESERVERWINDOW
 0000:0000  Imp  CREATEWINDOW         (USER.41)
 0002:1F86       DDEABANDONTRANSACTION
 0002:1BAC       DDEACCESSDATA
 0002:189A       DDEADDDATA
 0002:14B6       DDECLIENTTRANSACTION
 0002:1F3A       DDECMPSTRINGHANDLES
 0002:0C0E       DDECONNECT
 0002:07EE       DDECONNECTLIST
 0002:17EA       DDECREATEDATAHANDLE
 0002:1D08       DDECREATESTRINGHANDLE
 0002:0CA8       DDEDISCONNECT
 0002:0BA8       DDEDISCONNECTLIST
 0002:2186       DDEENABLECALLBACK
 0002:1CA0       DDEFREEDATAHANDLE
 0002:1DCA       DDEFREESTRINGHANDLE
 0002:1AB2       DDEGETDATA
 0002:17A6       DDEGETLASTERROR
 0002:0010       DDEINITIALIZE
 0002:1E36       DDEKEEPSTRINGHANDLE
 0002:22DC       DDENAMESERVICE
 0002:12B0       DDEPOSTADVISE
 0002:3362       DDEPOSTHOOKPROC
 0002:0F06       DDEQUERYCONVINFO
 0002:0AAC       DDEQUERYNEXTSERVER
 0002:1EA0       DDEQUERYSTRING
 0002:0D40       DDERECONNECT
 0002:326E       DDESENDHOOKPROC
 0002:11B8       DDESETUSERHANDLE
 0002:1C48       DDEUNACCESSDATA
 0002:044E       DDEUNINITIALIZE
 0000:0000  Imp  DEFHOOKPROC          (USER.235)
 0000:0000  Imp  DEFWINDOWPROC        (USER.107)
 0002:29D4       DELETEADVLIST
 0000:0000  Imp  DELETEDC             (GDI.68)
 0000:0000  Imp  DELETEMETAFILE       (GDI.127)
 0000:0000  Imp  DELETEOBJECT         (GDI.69)
 0002:67AC       DELETEQI
 0002:2534       DESTROYADVLST
 0002:27E0       DESTROYHWNDHSZLIST
 0002:24FC       DESTROYLST
 0002:2C64       DESTROYPILE
 0002:66D0       DESTROYQ
 0000:0000  Imp  DESTROYWINDOW        (USER.53)
 0000:0000  Imp  DIALOGBOX            (USER.87)
 0002:5462       DISCONNECT
 0000:0000  Imp  DISPATCHMESSAGE      (USER.114)
 0002:6D60       DLLENTRY
 0002:691C       DMGCREATEHEAP
 0002:695E       DMGDESTROYHEAP
 0002:3070       DMGDESTROYWINDOW
 0002:5A7E       DMGWNDPROC
 0002:5D42       DOCALLBACK
 0002:4CC6       DOCLIENTDDEMSG
 0002:64DA       EMPTYDDEPOSTQ
 0002:663E       EmptyQTimerProc
 0003:0146       EMPTYQUEUETIMERID
 0000:0000  Imp  ENDDIALOG            (USER.88)
 0000:0000  Imp  ENUMWINDOWS          (USER.54)
 0002:6A10       FARALLOCMEM
 0002:6A66       FARFREEMEM
 0002:5028       FEXPECTEDMSG
 0002:31EE       FINDADDHSZ
 0002:3214       FINDADDHSZHELPER
 0002:2A1C       FINDADVLIST
 0002:257A       FINDLSTITEM
 0002:2A4E       FINDNEXTADV
 0002:68AE       FINDNEXTQI
 0002:2CEE       FINDPILEITEM
 0002:6842       FINDQI
 0002:6C66       FREEDATAHANDLE
 0002:715A       FREEDDEDATA
 0002:3918       FREEDDEMSGDATA
 0002:30C0       FREEHSZ
 0000:0000  Imp  FREEPROCINSTANCE     (KERNEL.52)
 0003:003E       GATOMDDEMLMOM
 0003:0040       GATOMDMGCLASS
 0000:0000  Imp  GETCLASSWORD         (USER.129)
 0002:2428       GETCURRENTAPPINFO
 0000:0000  Imp  GETCURRENTTASK       (KERNEL.36)
 0000:0000  Imp  GETCURRENTTIME       (USER.15)
 0000:0000  Imp  GETDC                (USER.66)
 0002:72C0       GETDDECLIENTWINDOW
 0000:0000  Imp  GETDESKTOPWINDOW     (USER.286)
 0000:0000  Imp  GETKBCODEPAGE        (KEYBOARD.132)
 0000:0000  Imp  GETMESSAGE           (USER.108)
 0000:0000  Imp  GETMODULEUSAGE       (KERNEL.48)
 0000:0000  Imp  GETOBJECT            (GDI.82)
 0000:0000  Imp  GETPALETTEENTRIES    (GDI.363)
 0000:0000  Imp  GETPARENT            (USER.46)
 0000:0000  Imp  GETPROFILESTRING     (KERNEL.58)
 0000:0000  Imp  GETWINDOW            (USER.262)
 0000:0000  Imp  GETWINDOWLONG        (USER.135)
 0000:0000  Imp  GETWINDOWTASK        (USER.224)
 0000:0000  Imp  GETWINDOWWORD        (USER.133)
 0000:0000  Imp  GLOBALADDATOM        (USER.268)
 0000:0000  Imp  GLOBALALLOC          (KERNEL.15)
 0000:0000  Imp  GLOBALDELETEATOM     (USER.269)
 0000:0000  Imp  GLOBALFINDATOM       (USER.270)
 0000:0000  Imp  GLOBALFREE           (KERNEL.17)
 0000:0000  Imp  GLOBALGETATOMNAME    (USER.271)
 0000:0000  Imp  GLOBALLOCK           (KERNEL.18)
 0000:0000  Imp  GLOBALREALLOC        (KERNEL.16)
 0000:0000  Imp  GLOBALSIZE           (KERNEL.20)
 0000:0000  Imp  GLOBALUNLOCK         (KERNEL.19)
 0003:0042       GMESSAGEQUEUELIST
 0002:1C7A       HDDEDATA_VALIDATE
 0003:0018       HHEAPDMG
 0003:0016       HINSTANCE
 0000:0000  Imp  HMEMCPY              (KERNEL.348)
 0002:7D66       HUGEOFFSET
 0003:0024       HWINST
 0002:2826       HWNDFROMHSZ
 0002:30F8       INCHSZCOUNT
 0002:73DE       INITENUM
 0000:0000  Imp  INITTASK             (KERNEL.91)
 0000:0000  Imp  ISWINDOW             (USER.47)
 0000:0000  Imp  KILLTIMER            (USER.12)
 0001:0098       LIBENTRY
 0001:0000       LIBMAIN
 0000:0000  Imp  LOCALALLOC           (KERNEL.5)
 0000:0000  Imp  LOCALFREE            (KERNEL.7)
 0000:0000  Imp  LOCALHANDLE          (KERNEL.11)
 0000:0000  Imp  LOCALINIT            (KERNEL.4)
 0000:0000  Imp  LOCALSIZE            (KERNEL.10)
 0002:60A2       MAKECALLBACK
 0002:325A       MAKEINSTAPPNAME
 0000:0000  Imp  MAKEPROCINSTANCE     (KERNEL.51)
 0002:345A       MONBRDCASTCB
 0002:36F0       MONCONN
 0002:35C2       MONERROR
 0002:3530       MONHSZ
 0002:37D8       MONITORBROADCAST
 0002:389C       MONITORWNDPROC
 0002:3632       MONLINK
 0002:0050       MYATODW
 0002:2640       NEWLSTITEM
 0000:0000  Imp  OUTPUTDEBUGSTRING    (KERNEL.115)
 0003:001A       PAPPINFOLIST
 0000:0008  Abs  pAtomTable
 0003:001C       PDATAINFOPILE
 0000:0000  Imp  PEEKMESSAGE          (USER.109)
 0000:0006  Abs  pLocalHeap
 0003:0020       PLOSTACKPILE
 0002:2EC2       POPPILESUBITEM
 0002:619C       POSTDDEMESSAGE
 0000:0000  Imp  POSTMESSAGE          (USER.110)
 0000:0000  Imp  POSTQUITMESSAGE      (USER.6)
 0002:420E       POSTSERVERADVISE
 0003:003A       PREVHOOK
 0002:696E       PROCESSMEMERROR
 0002:7D12       PROCESSREGISTRATIONMESSAGE
 0000:000E  Abs  pStackBot
 0000:000C  Abs  pStackMin
 0000:000A  Abs  pStackTop
 0002:6B6E       PUTDATA
 0002:2CA0       QPILEITEMCOUNT
 0002:435A       QREPLY
 0002:314A       QUERYHSZLENGTH
 0002:3184       QUERYHSZNAME
 0002:6DDA       RECVPREP
 0002:00BE       REGISTER
 0000:0000  Imp  REGISTERCLASS        (USER.57)
 0002:6A8C       REGISTERCLASSES
 0002:7C34       REGISTERSERVICE
 0000:0000  Imp  REGISTERWINDOWMESSAGE (USER.118)
 0000:0000  Imp  RELEASEDC            (USER.68)
 0002:26F0       REMOVELSTITEM
 0003:0014       RMJ
 0003:0012       RMM
 0003:0004       rsrvptrs
 0003:0010       RUP
 0000:0000  Imp  SELECTOBJECT         (GDI.45)
 0002:3BDA       SENDCLIENTREQ
 0000:0000  Imp  SENDMESSAGE          (USER.111)
 0002:7B86       SENDMESSAGETOCLASS
 0002:787E       SERVERCREATE
 0002:7446       SERVERFRAMEINITCONV
 0002:3DBC       SERVERPROCESSDDEMSG
 0002:571C       SERVERWNDPROC
 0000:0000  Imp  SETPALETTEENTRIES    (GDI.364)
 0000:0000  Imp  SETPARENT            (USER.233)
 0000:0000  Imp  SETTIMER             (USER.10)
 0000:0000  Imp  SETWINDOWLONG        (USER.136)
 0000:0000  Imp  SETWINDOWSHOOK       (USER.121)
 0000:0000  Imp  SETWINDOWWORD        (USER.134)
 0003:0244       SHUTDOWNRETRYTIMEOUT
 0003:0248       SHUTDOWNTIMEOUT
 0003:0180       STKHQQ
 0002:59AC       SUBFRAMEWNDPROC
 0002:7D8E       SWITCHDS
 0003:005A       SZCLIENTCLASS
 0003:008A       SZCONVLISTCLASS
 0003:0050       SZDMGCLASS
 0003:0046       SZFRAMECLASS
 0003:009A       SZHEAPWATCHCLASS
 0003:007A       SZMONITORCLASS
 0003:0036       SZNULL
 0003:006A       SZSERVERCLASS
 0003:0230       SZT
 0002:040A       TERMDLGPROC
 0002:55B4       TERMINATE
 0002:5F00       TIMEOUT
 0000:0000  Imp  UNHOOKWINDOWSHOOK    (USER.234)
 0002:2476       UNLINKAPPINFO
 0002:3094       VALIDATEHCONV
 0001:0034       WEP
 0002:6DB6       XMITPREP
 0000:0000  Imp  YIELD                (KERNEL.29)
 0003:0230       _edata
 0003:024C       _end
 0000:0000  Imp  _wsprintf            (USER.420)
 0000:9876  Abs  __acrtmsg
 0000:9876  Abs  __acrtused
 0000:9876  Abs  __acrtused2
 0000:D6D6  Abs  __aDBdoswp
 0003:0182       __adbgmsg
 0003:0188       __aDBrterr
 0000:0000  Imp  __AHINCR             (KERNEL.114)
 0002:7DA4       __aNFaulshr
 0002:7DC2       __aNulshr
 0003:0198       __caption
 0003:0230       __edata
 0003:024C       __end
 0000:9876  Abs  __fptaskdata
 0002:7DCE       __NMSG_TEXT
 0002:7DF9       __NMSG_WRITE
 0002:7DA1       __wflags
 0000:0000  Imp  __WINFLAGS           (KERNEL.178)
 0003:018A       ___aDBexit
 0003:0186       ___aDBswpchk
 0003:0184       ___aDBswpflg

  Address         Publics by Value

 0000:0000  Imp  _wsprintf            (USER.420)
 0000:0000  Imp  DIALOGBOX            (USER.87)
 0000:0000  Imp  DEFWINDOWPROC        (USER.107)
 0000:0000  Imp  GLOBALDELETEATOM     (USER.269)
 0000:0000  Imp  REGISTERWINDOWMESSAGE (USER.118)
 0000:0000  Imp  GLOBALFREE           (KERNEL.17)
 0000:0000  Imp  GLOBALSIZE           (KERNEL.20)
 0000:0000  Imp  RELEASEDC            (USER.68)
 0000:0000  Imp  GETDESKTOPWINDOW     (USER.286)
 0000:0000  Imp  GETPARENT            (USER.46)
 0000:0000  Imp  CREATECOMPATIBLEBITMAP (GDI.51)
 0000:0000  Imp  LOCALHANDLE          (KERNEL.11)
 0000:0000  Imp  ENUMWINDOWS          (USER.54)
 0000:0000  Imp  ISWINDOW             (USER.47)
 0000:0000  Imp  DISPATCHMESSAGE      (USER.114)
 0000:0000  Imp  GETPROFILESTRING     (KERNEL.58)
 0000:0000  Imp  GETCLASSWORD         (USER.129)
 0000:0000  Imp  DELETEMETAFILE       (GDI.127)
 0000:0000  Imp  CREATEWINDOW         (USER.41)
 0000:0000  Imp  DEFHOOKPROC          (USER.235)
 0000:0000  Imp  GETMODULEUSAGE       (KERNEL.48)
 0000:0000  Imp  POSTQUITMESSAGE      (USER.6)
 0000:0000  Imp  FREEPROCINSTANCE     (KERNEL.52)
 0000:0000  Imp  POSTMESSAGE          (USER.110)
 0000:0000  Imp  GLOBALFINDATOM       (USER.270)
 0000:0000  Imp  REGISTERCLASS        (USER.57)
 0000:0000  Imp  __WINFLAGS           (KERNEL.178)
 0000:0000  Imp  YIELD                (KERNEL.29)
 0000:0000  Imp  LOCALALLOC           (KERNEL.5)
 0000:0000  Imp  SETPALETTEENTRIES    (GDI.364)
 0000:0000  Imp  GETPALETTEENTRIES    (GDI.363)
 0000:0000  Imp  SETTIMER             (USER.10)
 0000:0000  Imp  SETWINDOWSHOOK       (USER.121)
 0000:0000  Imp  CREATEPALETTE        (GDI.360)
 0000:0000  Imp  GETWINDOWLONG        (USER.135)
 0000:0000  Imp  SETWINDOWLONG        (USER.136)
 0000:0000  Imp  HMEMCPY              (KERNEL.348)
 0000:0000  Imp  SENDMESSAGE          (USER.111)
 0000:0000  Imp  ENDDIALOG            (USER.88)
 0000:0000  Imp  BITBLT               (GDI.34)
 0000:0000  Imp  PEEKMESSAGE          (USER.109)
 0000:0000  Imp  GETDC                (USER.66)
 0000:0000  Imp  UNHOOKWINDOWSHOOK    (USER.234)
 0000:0000  Imp  SELECTOBJECT         (GDI.45)
 0000:0000  Imp  GETWINDOW            (USER.262)
 0000:0000  Imp  LOCALFREE            (KERNEL.7)
 0000:0000  Imp  COPYMETAFILE         (GDI.151)
 0000:0000  Imp  GETWINDOWWORD        (USER.133)
 0000:0000  Imp  SETWINDOWWORD        (USER.134)
 0000:0000  Imp  GLOBALLOCK           (KERNEL.18)
 0000:0000  Imp  GLOBALUNLOCK         (KERNEL.19)
 0000:0000  Imp  KILLTIMER            (USER.12)
 0000:0000  Imp  GETWINDOWTASK        (USER.224)
 0000:0000  Imp  CALLMSGFILTER        (USER.123)
 0000:0000  Imp  GLOBALGETATOMNAME    (USER.271)
 0000:0000  Imp  GETCURRENTTIME       (USER.15)
 0000:0000  Imp  GETKBCODEPAGE        (KEYBOARD.132)
 0000:0000  Imp  GETOBJECT            (GDI.82)
 0000:0000  Imp  CREATECOMPATIBLEDC   (GDI.52)
 0000:0000  Imp  GETCURRENTTASK       (KERNEL.36)
 0000:0000  Imp  DESTROYWINDOW        (USER.53)
 0000:0000  Imp  LOCALINIT            (KERNEL.4)
 0000:0000  Imp  DELETEDC             (GDI.68)
 0000:0000  Imp  SETPARENT            (USER.233)
 0000:0000  Imp  DELETEOBJECT         (GDI.69)
 0000:0000  Imp  LOCALSIZE            (KERNEL.10)
 0000:0000  Imp  GETMESSAGE           (USER.108)
 0000:0000  Imp  OUTPUTDEBUGSTRING    (KERNEL.115)
 0000:0000  Imp  __AHINCR             (KERNEL.114)
 0000:0000  Imp  GLOBALALLOC          (KERNEL.15)
 0000:0000  Imp  GLOBALREALLOC        (KERNEL.16)
 0000:0000  Imp  INITTASK             (KERNEL.91)
 0000:0000  Imp  GLOBALADDATOM        (USER.268)
 0000:0000  Imp  MAKEPROCINSTANCE     (KERNEL.51)
 0000:0006  Abs  pLocalHeap
 0000:0008  Abs  pAtomTable
 0000:000A  Abs  pStackTop
 0000:000C  Abs  pStackMin
 0000:000E  Abs  pStackBot
 0000:9876  Abs  __acrtused
 0000:9876  Abs  __acrtused2
 0000:9876  Abs  __fptaskdata
 0000:9876  Abs  __acrtmsg
 0000:D6D6  Abs  __aDBdoswp
 0001:0000       LIBMAIN
 0001:0034       WEP
 0001:0098       LIBENTRY
 0002:0010       DDEINITIALIZE
 0002:0050       MYATODW
 0002:00BE       REGISTER
 0002:040A       TERMDLGPROC
 0002:044E       DDEUNINITIALIZE
 0002:07EE       DDECONNECTLIST
 0002:0AAC       DDEQUERYNEXTSERVER
 0002:0BA8       DDEDISCONNECTLIST
 0002:0C0E       DDECONNECT
 0002:0CA8       DDEDISCONNECT
 0002:0D40       DDERECONNECT
 0002:0F06       DDEQUERYCONVINFO
 0002:11B8       DDESETUSERHANDLE
 0002:12B0       DDEPOSTADVISE
 0002:14B6       DDECLIENTTRANSACTION
 0002:17A6       DDEGETLASTERROR
 0002:17EA       DDECREATEDATAHANDLE
 0002:189A       DDEADDDATA
 0002:1AB2       DDEGETDATA
 0002:1BAC       DDEACCESSDATA
 0002:1C48       DDEUNACCESSDATA
 0002:1C7A       HDDEDATA_VALIDATE
 0002:1CA0       DDEFREEDATAHANDLE
 0002:1D08       DDECREATESTRINGHANDLE
 0002:1DCA       DDEFREESTRINGHANDLE
 0002:1E36       DDEKEEPSTRINGHANDLE
 0002:1EA0       DDEQUERYSTRING
 0002:1F3A       DDECMPSTRINGHANDLES
 0002:1F86       DDEABANDONTRANSACTION
 0002:2050       ABANDONTRANSACTION
 0002:2186       DDEENABLECALLBACK
 0002:22DC       DDENAMESERVICE
 0002:2428       GETCURRENTAPPINFO
 0002:2476       UNLINKAPPINFO
 0002:24BC       CREATELST
 0002:24FC       DESTROYLST
 0002:2534       DESTROYADVLST
 0002:257A       FINDLSTITEM
 0002:25DA       CMPDWORD
 0002:2602       CMPWORD
 0002:2620       CMPHIWORD
 0002:2640       NEWLSTITEM
 0002:26F0       REMOVELSTITEM
 0002:27A0       ADDHWNDHSZLIST
 0002:27E0       DESTROYHWNDHSZLIST
 0002:2826       HWNDFROMHSZ
 0002:285E       CMPADV
 0002:28EE       COUNTADVREQLEFT
 0002:2956       ADDADVLIST
 0002:29D4       DELETEADVLIST
 0002:2A1C       FINDADVLIST
 0002:2A4E       FINDNEXTADV
 0002:2AA6       CLEANUPADVLIST
 0002:2C10       CREATEPILE
 0002:2C64       DESTROYPILE
 0002:2CA0       QPILEITEMCOUNT
 0002:2CEE       FINDPILEITEM
 0002:2DD8       ADDPILEITEM
 0002:2EC2       POPPILESUBITEM
 0002:2F62       COPYHUGEBLOCK
 0002:3070       DMGDESTROYWINDOW
 0002:3094       VALIDATEHCONV
 0002:30C0       FREEHSZ
 0002:30F8       INCHSZCOUNT
 0002:314A       QUERYHSZLENGTH
 0002:3184       QUERYHSZNAME
 0002:31EE       FINDADDHSZ
 0002:3214       FINDADDHSZHELPER
 0002:325A       MAKEINSTAPPNAME
 0002:326E       DDESENDHOOKPROC
 0002:3362       DDEPOSTHOOKPROC
 0002:345A       MONBRDCASTCB
 0002:3530       MONHSZ
 0002:35C2       MONERROR
 0002:3632       MONLINK
 0002:36F0       MONCONN
 0002:37D8       MONITORBROADCAST
 0002:383C       ALLOCMONBUF
 0002:389C       MONITORWNDPROC
 0002:3918       FREEDDEMSGDATA
 0002:398C       CLIENTXFERREQ
 0002:3BDA       SENDCLIENTREQ
 0002:3DBC       SERVERPROCESSDDEMSG
 0002:420E       POSTSERVERADVISE
 0002:435A       QREPLY
 0002:4764       CLIENTXFERRESPOND
 0002:4A20       CLIENTWNDPROC
 0002:4CC6       DOCLIENTDDEMSG
 0002:5028       FEXPECTEDMSG
 0002:50FC       ADVANCEXACTION
 0002:52F4       CHECKCBQ
 0002:5462       DISCONNECT
 0002:55B4       TERMINATE
 0002:571C       SERVERWNDPROC
 0002:59AC       SUBFRAMEWNDPROC
 0002:5A12       CHILDMSG
 0002:5A7E       DMGWNDPROC
 0002:5C46       CONVLISTWNDPROC
 0002:5D42       DOCALLBACK
 0002:5F00       TIMEOUT
 0002:605C       ALLOCDDESEL
 0002:60A2       MAKECALLBACK
 0002:619C       POSTDDEMESSAGE
 0002:64DA       EMPTYDDEPOSTQ
 0002:663E       EmptyQTimerProc
 0002:6666       CREATEQ
 0002:66D0       DESTROYQ
 0002:66EC       ADDQI
 0002:67AC       DELETEQI
 0002:6842       FINDQI
 0002:68AE       FINDNEXTQI
 0002:691C       DMGCREATEHEAP
 0002:695E       DMGDESTROYHEAP
 0002:696E       PROCESSMEMERROR
 0002:6A10       FARALLOCMEM
 0002:6A66       FARFREEMEM
 0002:6A8C       REGISTERCLASSES
 0002:6B6E       PUTDATA
 0002:6C66       FREEDATAHANDLE
 0002:6D60       DLLENTRY
 0002:6DB6       XMITPREP
 0002:6DDA       RECVPREP
 0002:6E60       COPYDDESHAREHANDLE
 0002:6EB2       COPYBITMAP
 0002:6F8A       COPYPALETTE
 0002:7022       COPYHDDEDATA
 0002:715A       FREEDDEDATA
 0002:71F8       CLIENTCREATE
 0002:72C0       GETDDECLIENTWINDOW
 0002:73DE       INITENUM
 0002:7446       SERVERFRAMEINITCONV
 0002:77CA       CREATESERVERWINDOW
 0002:787E       SERVERCREATE
 0002:78F2       CLIENTINITACK
 0002:7B86       SENDMESSAGETOCLASS
 0002:7C34       REGISTERSERVICE
 0002:7D12       PROCESSREGISTRATIONMESSAGE
 0002:7D66       HUGEOFFSET
 0002:7D8E       SWITCHDS
 0002:7DA1       __wflags
 0002:7DA4       __aNFaulshr
 0002:7DC2       __aNulshr
 0002:7DCE       __NMSG_TEXT
 0002:7DF9       __NMSG_WRITE
 0003:0004       rsrvptrs
 0003:0010       RUP
 0003:0012       RMM
 0003:0014       RMJ
 0003:0016       HINSTANCE
 0003:0018       HHEAPDMG
 0003:001A       PAPPINFOLIST
 0003:001C       PDATAINFOPILE
 0003:0020       PLOSTACKPILE
 0003:0024       HWINST
 0003:0026       CCDEF
 0003:0036       SZNULL
 0003:0038       CMONITOR
 0003:003A       PREVHOOK
 0003:003E       GATOMDDEMLMOM
 0003:0040       GATOMDMGCLASS
 0003:0042       GMESSAGEQUEUELIST
 0003:0046       SZFRAMECLASS
 0003:0050       SZDMGCLASS
 0003:005A       SZCLIENTCLASS
 0003:006A       SZSERVERCLASS
 0003:007A       SZMONITORCLASS
 0003:008A       SZCONVLISTCLASS
 0003:009A       SZHEAPWATCHCLASS
 0003:00AC       APROGMANHACK
 0003:00AE       AULMAPTYPE
 0003:0146       EMPTYQUEUETIMERID
 0003:0180       STKHQQ
 0003:0182       __adbgmsg
 0003:0184       ___aDBswpflg
 0003:0186       ___aDBswpchk
 0003:0188       __aDBrterr
 0003:018A       ___aDBexit
 0003:0198       __caption
 0003:0230       _edata
 0003:0230       __edata
 0003:0230       SZT
 0003:0244       SHUTDOWNRETRYTIMEOUT
 0003:0248       SHUTDOWNTIMEOUT
 0003:024C       __end
 0003:024C       _end

Program entry point at 0001:0098
